:1000000000308A008F2900000A108A100A11820726
:100010002934003430340034373400343F30840025
:100020000008031925280230F800BF30F7006400EB
:10003000F70B1728F80B15289630F700F70B1E283A
:10004000000000006400800B13288A11402808304B
:10005000BF02031C36283F3084000310800C0008C8
:100060000319362834286400800B33288A1143286A
:10007000831605118312051564000130BF000E2898
:10008000C730BF0027282408BE00BE0803194A282D
:10009000BE03452883160511831205113830AE00C2
:1000A0000030AF008A11362A0034A81B7D28A8082A
:1000B000031D5E282708003C03187D280108801FC7
:1000C0006428A81F6C286628A81B7528A808031D8B
:1000D0006C282702031C7528831685138312851349
:1000E00083160513831205177D28831605138312C3
:1000F00005138316851383128513A708031D87280C
:10010000A808031D87288316051383120513831679
:10011000851383128513A81FBD280108C000280875
:10012000FA002708A81F9D282708003CF700FA01BD
:100130002808031C280FFA027708F800C01FA3281C
:10014000FA1FAC28A528FA1BB528FA08031DAC280D
:1001500040087802031CB528831605138312051383
:100160008316851383128517BD2883160513831202
:1001700005138316851383128513A61BE528A6088D
:10018000031DC6282508003C0318E5280108801F28
:10019000CC28A61FD428CE28A61BDD28A608031D20
:1001A000D4282502031CDD288316851083128510B0
:1001B0008316051083120514E52883160510831293
:1001C00005108316851083128510A508031DEF28DE
:1001D000A608031DEF288316051083120510831649
:1001E000851083128510A61F25290108C000260846
:1001F000FA002508A61F05292508003CF700FA018A
:100200002608031C260FFA027708F800C01F0B29E6
:10021000FA1F14290D29FA1B1D29FA08031D142998
:1002200040087802031C1D2983160510831205104F
:1002300083168510831285142529831605108312D1
:10024000051083168510831285105530B5000030D7
:10025000B6008A11362A0034130893018316141845
:10026000332983122E2983121308A1008316061046
:10027000831206148316061083120610211C4829C7
:10028000BE30A400A601A501A8017F30A7002C293B
:10029000211F52293C30A400A801A701A6017F30EC
:1002A000A5002C29A11C5D299E30A400A601463082
:1002B000A500A8017F30A7002C29A11E6829623063
:1002C000A400A8014630A700A6017F30A5002C2974
:1002D000211D73299430A400A6015A30A500A8015D
:1002E0007F30A7002C29211E7E296C30A400A80194
:1002F0005A30A700A6017F30A5002C29A11D88290E
:100300008030A400A6016430A500A801A7002C2914
:100310002C30BC000130BD008A11362A0034840123
:100320001F308305703083168F001F129F121B0829
:1003300080399B0007309C001F129F121B088039D8
:100340009B001F1383121F179F1783169F1383127F
:100350001F1494128316061186140612303083126D
:1003600094000030831694000108C73908388100D2
:1003700083129001723083168F00051383120513C8
:1003800083168513831285138316051083120510B7
:1003900083168510831285108030A400A601A50164
:1003A000A801A701A901AB010830AA00AD010130E5
:1003B000AC003830AE000030AF00B001B201013007
:1003C000B100B401B3015530B5000030B600B7013B
:1003D000B9010230B800BB01BA012C30BC000130B9
:1003E000BD00A0010030F80006389200FA308316F4
:1003F000920083128C100030F80006389200FA3018
:100400008316920083128C100310200DF700042035
:10041000F900013077070420FA0079088400000809
:10042000F900840A0008F700840A0008F800840A2A
:10043000800A0008FA00031D202A840A800A840327
:10044000840A00087802031D382A77087A02031DFF
:10045000382A84038001840A8001840AF91B382A1F
:10046000840A00088A0084030008820083120313B0
:10047000A00A03302002031D042AA0018C1C422A7A
:0C0480008316022A3E2AFF30A000630011
:04400E00F83FFF3F39
:00000001FF
